:103800000C942A1C0C94471C0C94471C0C94471CC9
:103810000C94471C0C94471C0C94471C0C94471C9C
:103820000C94471C0C94471C0C94471C0C94471C8C
:103830000C94471C0C94471C0C94471C0C94471C7C
:103840000C94471C0C94471C0C94471C0C94471C6C
:103850000C94471C11241FBECFE5D4E0DEBFCDBFC2
:1038600010E0A0E6B0E0E0E0FFE302C005900D92BA
:10387000A036B107D9F711E0A0E6B0E001C01D9273
:10388000A43AB107E1F70E94371F0C947E1F0C94F5
:10389000001C0F92AF93BF93CF93DF93EF93FF93EF
:1038A000FC01EA01DB01C895099231961197D9F71D
:1038B000FF91EF91DF91CF91BF91AF910F9008955C
:1038C0000F921F920F931F93AF93BF93CF93DF93EA
:1038D000EF93FF93FC01EA01DB0110E809901990D6
:1038E00001E04CD03296129711F01250B9F7FC015A
:1038F00003E044D005E042D000E810E0800F911FC3
:10390000109759F7FF91EF91DF91CF91BF91AF9150
:103910001F910F911F900F9008950F931F93EF9396
:10392000FF93FC0103E02AD000E810E0E00FF11F54
:10393000E617F707B9F7FF91EF911F910F910895DF
:103940000F930F9222D0082E09E018D00F900F91FC
:1039500008950F930F92EF93FF9317D0FC0160939C
:103960005700C895802DFF91EF910F900F9108950A
:103970000F930BD001E102D00F910895E199FECF92
:1039800000935700E895FFFF00000091570000FDED
:10399000FCCF089589E089B98AB188618AB9089510
:1039A0008AB1877E8AB908958CB95E9BFECF5E9AF4
:1039B00008958CB108958BB180780895AC0120E012
:1039C00030E009C05F9BFECF8CB1FA01E20FF31F1C
:1039D00080832F5F3F4F26173707A0F381E00895BC
:1039E000FC0120E030E008C080818CB95E9BFECFF6
:1039F00031965E9A2F5F3F4F26173707A8F381E075
:103A00000895813879F0823818F4803839F408C084
:103A1000823851F0883911F483E0089580E00895E8
:103A200082E0089581E0089582E108956091A00008
:103A30007091A1004091A2015091A30120E030E0DB
:103A400010C0C901840F951F9FBB8EBBF901EE55B5
:103A5000FF4F80818DBBE29AE19AE199FECF2F5F03
:103A60003F4F2617370768F3460F571F5093A301A0
:103A70004093A20108956091A0007091A10040912F
:103A8000A2015091A30120E030E00DC0C901840FD4
:103A9000951F9FBB8EBBE09A8DB3F901EE55FF4F8A
:103AA00080832F5F3F4F2617370780F3460F571F3E
:103AB0005093A3014093A201089540E050E00BC051
:103AC00020E030E000002F5F3F4F68E02A3C3607DF
:103AD000C9F74F5F5F4F4817590790F308956091FA
:103AE000A0007091A1008091A2019091A30142EAEF
:103AF00050E0880F991F0E94491C0895CF93DF93CF
:103B0000C0E0D0E011C0AE014E555F4F8091A201E0
:103B10009091A301880F991F60E870E08C0F9D1FA2
:103B20000E94601CC058DF4F8091A0009091A100BE
:103B3000C817D90740F30E94B81CDF91CF910895B0
:103B40000E94DB1C8823E1F30E94D91C803211F40F
:103B500081E0089585E10E94D41C80E00895DF9201
:103B6000EF92FF920F931F93CF93DF9369E081E071
:103B700090E00E94A91C84FF03C08F7E0E94A01CBD
:103B8000DD240E94DB1C8823E1F30E94D91C8235CE
:103B9000C0F4803508F079C0813409F443C0823420
:103BA00048F4813321F1803409F453C1803309F0A2
:103BB0004CC16BC0823409F459C0853409F045C149
:103BC00058C0863509F40EC1873538F4823509F4BA
:103BD00062C0853509F039C16DC0843709F4A7C0CA
:103BE000853709F4EFC0843609F02FC17BC00E94ED
:103BF000A01D882331F284E10E94D41C81E40E943C
:103C0000D41C86E50E94D41C82E50E94D41C80E26C
:103C10000E94D41C83E50E94D41C84E50E94D41C1D
:103C20008BE40FC161E070E080E690E00E94DE1C52
:103C30000E94A01D882309F4A4CF84E10E94D41C13
:103C400080916000813871F0823818F4803831F446
:103C500007C0823849F0883909F4C2C080E0F1C059
:103C600082E0EFC081E0EDC082E1EBC064E170E092
:103C700008C061E070E080E690E00E94DE1C64E035
:103C800070E080E690E00E94DE1C0E94A01D882368
:103C900009F477CF0DC00E94A01D882309F471CFCD
:103CA00060E070E480E090E00E948D1C0E94B81CEF
:103CB00084E1C7C062E070E080E690E00E94DE1C14
:103CC0000E94A01D882309F45CCFF0906100EE24CF
:103CD000809160009701280F311D3093A30120933C
:103CE000A201E6CF63E070E080E690E00E94DE1C77
:103CF000D0916000C0E080916100BE01680F711D2D
:103D00007093A1006093A00082EA90E00E94DE1C04
:103D10000E94A01D882309F434CF8091620086346C
:103D200019F40E947E1DC4CF0E94161DC1CF63E00E
:103D300070E080E690E00E94DE1C1091600000E0E0
:103D4000809161009801280F311D3093A1002093CC
:103D5000A0000E94A01D882309F413CF8091620067
:103D6000863459F04091A0005091A1006091A201C9
:103D70007091A30120E030E010C00E946F1D16C0BA
:103D8000C901860F971F9FBB8EBBE09A8DB3F901C7
:103D9000EE55FF4F80832F5F3F4F2417350780F389
:103DA000460F571F5093A3014093A20184E10E9444
:103DB000D41C6091A0007091A10082EA90E00E9462
:103DC000F01C41C00E94A01D882309F4DACE84E1D2
:103DD0000E94D41C8EE10E94D41C84E90E94D41C51
:103DE00083E02FC064E070E080E690E00E94DE1C7B
:103DF0000E94A01D882309F4C4CE84E10E94D41C33
:103E000080916000803531F480916100882359F4FD
:103E1000DD2412C0883581F480916100883041F43E
:103E200053E0D52E09C0883039F442E0D42E04C0C6
:103E3000882311F4DD24D39469E08D2D90E00E9455
:103E4000A91C0E94D41C80E101C085E10E94D41C01
:103E500098CEDF91CF911F910F91FF90EF90DF905F
:103E600008950E94D01CE0E0F0E0099508951F93AA
:103E7000F894E199FECF8EEF91E09FBB8EBBE09A64
:103E80008DB3843B99F4E199FECF8FEF91E09FBB16
:103E90008EBBE09A8DB3833C49F4E199FECF8DEF60
:103EA00091E09FBB8EBBE09A8DB381BF0E94CA1C7C
:103EB0000E94D91C1EE119C00000019648E08A3C0E
:103EC0009407D1F72F5F3F4F2436310519F080E07A
:103ED00090E0F2CF0E94DB1C882319F00E94AF1DF6
:103EE00007C0115018BB112319F020E030E0EFCFCC
:103EF0000E94311F80E090E01F910895F894FFCF59
:0400000300003800C1
:00000001FF
